:020000040000FA
:1000000025003A0C26000A0C06003A0C06000000F7
:1000100006023800300E3A0D060066093900830CDE
:1000200002004604700058092607130A15029400BE
:100030003800F50110024306250A3E0C980003071C
:10004000110A640C98000306110A58092606250AAD
:100050001502940038000C0C98000307110A5D0C7F
:1000600098000306110A280C98001002180F430686
:100070003E0AB002710372037303130A46050306B6
:100080003A0A1302150F43073A0A1202990143076D
:100090003A0A1102570F4306520A030F43073A0A5E
:1000A0000604110A0605700C3600720C3700110A9E
:1000B00014028100F4010307000804000607010888
:1000C000F6004306F7004306060402089803030EF1
:0A00D000E201540815084508510824
:080400000500040005000000E6
:021FFE00FE0FD4
:00000001FF
